:100000000BC018951895189518957CC018951895DB
:1000100018951895189518958FED8DBFC6EDEAEDDA
:100020004E2EDD275D2EA89584B7082E877F84BFCE
:1000300088E1992781BD91BDEEE7F0E0A0E6B0E050
:1000400088278D933197E9F76624D49AB89A80E08F
:1000500080BF89E88FBD73E27BBD8FB5807F8FBD88
:10006000789479B7746079BFDC9AC09A709168000F
:1000700070627093680081E080936400A8E68C91C0
:1000800086FB0EF407C0A6E38C9186FBA5E68827C5
:1000900080F98C934091640000916500041709F485
:1000A00030C0A5E68C9180FBA8E68C9187F98C93F3
:1000B0008091650080936400C09ADC9A709168001A
:1000C00070647093680084E180936600A8E68C9168
:1000D00085FB0EF004C084E68093630003C085E6D0
:1000E0008093630001E440916600040F0BBD0BB5E3
:1000F00040916600040F0BBD80E08093670089E8A3
:100100008FBDBCCF0F921F922F923F924F925F9262
:100110007F92AF92BF920F931F932F933F934F9372
:100120005F936F937F938F939F93AF93BF93CF937F
:10013000DF93EF93FF938FB78F93A8E68C9187FBA4
:100140000EF40FC0A2E68C918F5F8C930091620039
:10015000033010F009F001C003C080E0809362001A
:100160000DC0809162008150809362000091620016
:100170000F3F09F003C083E080936200E4E8F2E0FF
:10018000A2E68C919927A0E6A7D00BB340EF0423F9
:10019000A1E60C930091610040916000042B0BBB21
:1001A00000916700003009F01AC00091660000302D
:1001B00010F009F001C00CC080916600815080935E
:1001C00066008BB58A958BBD8BB58A958BBD06C0B5
:1001D00081E08093670084E18093660016C001305F
:1001E00009F013C04091660000916300041710F0FD
:1001F00009F00BC0A8E68C9185FB0EF406C08BB508
:1002000083958BBD8BB583958BBD809163008150A9
:100210008093630000916300003009F017C0709173
:1002200068007F7D709368008FB5807F8FBDC09818
:1002300084EF91E032D0709168007F7B709368000A
:10024000A8E68C9187FB0EF401C0DC988F918FBFDC
:10025000FF91EF91DF91CF91BF91AF919F918F91DE
:100260007F916F915F914F913F912F911F910F91CE
:10027000BF90AF907F905F904F903F902F901F90D6
:100280000F9018950A0905063197F1F708956894BB
:1002900062F80895E89462F80895EF93FF93EE27CB
:1002A000E82BE92B31F0E0EDF7E03197F1F701971A
:1002B000D1F7FF91EF910895C895319600200895E8
:1002C00091E005C092E003C094E001C098E0F4DF43
:0E02D0000D929A95E1F70895E80FF91FF1CF0E
:00000001FF
